:10000000FFEF01F00000000000EF00F00000000032
:0A0010000000000000000000F3D71C
:06001C00000000001200CC
:10002200120E0C6EDA0E0D6E0D2EFED70C2EFCD7B4
:0400320000001200B8
:0C003600290E0D6E0D2EFED700001200EA
:100042000001B5BF02D0819E01D0818EB5BD02D024
:10005200819C01D0818CB5BB02D0819A01D0818A6A
:10006200B5B902D0819801D081888EB102D0818445
:1000720001D081948186D1DF8196B5B702D0819E6D
:1000820001D0818EB5B502D0819C01D0818CB5B3EF
:1000920002D0819A01D0818AB5B102D0819801D073
:1000A20081888EB102D0818401D081948186B5DFAE
:0E00B20081968EA102D0B4DF01D0BCDF120017
:0E00C000ACB202D00000FCD7B4C0ADFF1200FD
:0E00CE0000018E91B4C0B5F0B5DF8E81120036
:0A00DC00120E0D6E0D2EFED712005D
:1000E600086A096A100E0C6E013408360936045087
:1000F600085E0550D8A0053C095ED8B007D004506C
:1001060008260550D8B0053C0926D8900036013699
:060116000C2EEAD71200D6
:10011C00C26A070EC012C08EADC000F0003600904F
:10012C00003600900050C212C280D2DFC282C2A23E
:10013C0001D0FDD7C4CF01F0006AC3500012000EED
:06014C000112C290120036
:100152000001B16B050EB15D0AE2B151AF25E16E4E
:10016200000EB021E26E200EE66EB12BF3D7B15134
:10017200AF25E16E000EB021E26EE66AB107B15121
:10018200AF25B26F000EB021B36F0A0E046E000EDF
:10019200056EADC000F0AEC001F0A4DF08C000F0F3
:1001A20009C001F0300E0026B2C0E1FFB3C0E2FF89
:1001B20000C0E6FF0A0E046E000E056EADC000F030
:1001C200AEC001F08FDF00C0ADF001C0AEF0000E96
:1001D200011802E1000E001801E102D0B107CFD7E9
:0201E200120009
:0A01E400000EACB2010E006E120016
:1001EE000001B06BADC0E9FFAEC0EAFFEECFAFF0DD
:1001FE00AF51000A0EE0AFC0B4F05BDF0001B02BD0
:10020E00B051AD25E96E000EAE21EA6EEECFAFF025
:04021E00EFD7120004
:10022200C00E0001976F000E986FB40E996F000E0A
:100232009A6FFF0E936FFF0E946F000E956F000E74
:10024200966FFF0E8F6FFF0E906F000E916F000E74
:10025200926FE40E886F010E896F000E8A6F000E96
:100262008B6FAC8A900EAB6E948E949C9EAA03D038
:08027200AECF00F0FBD7120033
:10027A000900F5CFE6FF0006FBE10106F9E11200ED
:10028A000D0E0001B46F17DF0A0E0001B46F13DF01
:02029A00120050
:10029C0010D0800E0001AD6F1AD0C00EAD6F17D00C
:1002AC00940EAD6F14D0D40EAD6F11D0800EAD6F17
:1002BC000ED00001AD51010AECE0AD51020AEDE0A7
:1002CC00AD51030AEDE0AD51040AEDE0EFD7AE05F8
:1002DC00006EAD51002600C0ADF000C0B5F0ABDE35
:1002EC008E91B16BB151AF25E96E000EB021EA6E63
:1002FC00EE520BE0B151AF25E96E000EB021EA6E63
:0E030C00EECFB4F0DEDEB12BEDD78E81120005
:10031A00C30EC216ADC000F0003600900036009041
:10032A000050C212D6DEC282C2A201D0FDD7C4CF0B
:0E033A0001F0006AC3500012000E0112120002
:100348001A0E0001A76F030EA86FAD0EA96F000E5D
:0E035800AA6FC26A070EC012C08EC2801200C9
:10036600939693949398939A939C939E8196819453
:10037600819E819C819A819851DE50DE4FDE818A72
:100386008188818648DE819649DE818644DE8196B3
:1003960045DE818640DE819641DE819881863BDEA0
:1003A60081963CDE818637DE8196819A818E8186B2
:1003B60032DE819633DE819E818881862CDE8196AF
:1003C6008198818628DE819629DE818624DE8196C3
:1003D6008188818620DE819621DE819881861BDEDA
:1003E6008196818E818C818A8188818614DE8196B0
:0803F60015DE00018E811200EA
:1003FE0040EC03F07F6A010E7E6E7B9E7A9E936ABE
:10040E00EF0E926EBD0E946EB886B06A810EAF6E10
:10041E00AC8400DF010EC26EC16AC08EC08AC09865
:10042E00C096C094C082C090D6DE0050000A01E192
:10043E00FBD70C0E0001B46F3CDE070E0B6E580E90
:10044E000C6E590E0D6E0D2EFED70C2EFCD70B2EEC
:10045E00FAD7000000006C0E0001AD6F000EAE6FFB
:10046E00BFDE6BDF79DF020E0B6E450E0C6EA90E32
:10047E000D6E0D2EFED70C2EFCD70B2EFAD70000CC
:10048E000000010EB56FD6DD0C0EB56FD3DD010E7B
:10049E00AD6F010EAE6F5B0EAF6F000EB06FF7DE7D
:1004AE00020EAD6F010EAE6F310EAF6F000EB06F5C
:1004BE00EEDE330E0B6EBB0E0C6EDF0E0D6E0D2EC2
:1004CE00FED70C2EFCD70B2EFAD700000000150E0F
:1004DE00AD6F000EAE6F84DE010EB56FABDD010E9B
:1004EE00AD6F010EAE6F4A0EAF6F000EB06FCFDE66
:1004FE000D0E0B6EAF0E0C6EB60E0D6E0D2EFED7D4
:10050E000C2EFCD70B2EFAD700008C6B8D6B010EC8
:10051E00B56F90DD010EAD6F010EAE6F420EAF6F77
:10052E00000EB06FB4DE8CC0ADF08DC0AEF09B0E81
:10053E00AF6F000EB06F06DE9B0EAD6F000EAE6F8E
:10054E004FDE080EB46FB5DD010E0001AD6F080E63
:10055E00AE6F9B0EAF6F000EB06F99DEAD6BD7DD39
:10056E0000C0ABF001C0ACF000C0ADF001C0AEF009
:10057E009B0E0001AF6F000EB06FE4DD9B0EAD6FF2
:10058E00000EAE6F2DDE080EB46F93DD020E00016D
:10059E00AD6FBCDE00C0ABF001C0ACF000C0ADF082
:1005AE0001C0AEF09B0E0001AF6F000EB06FCADD42
:1005BE009B0EAD6F000EAE6F13DE020EAD6F010E11
:1005CE00AE6F9B0EAF6F000EB06F61DE070E0B6E3F
:1005DE00580E0C6E590E0D6E0D2EFED70C2EFCD72E
:1005EE000B2EFAD70000000080A802D0809801D010
:0E05FE00808844DE00018C4B8D2B8CD7FFD7FC
:1006800010EE15F0730E006E010E016E0C0EF66E7C
:0E069000060EF76E000EF86E3DEC01F0120043
:10060C004C6574277320676F20666F7220414443DA
:0C061C00206D656173757265200A0D0089
:100628007769746820626F6F746C6F61646572209B
:0106380000C1
:080639004D6573757265200028
:10064100434F4720203278313620626F6172642037
:0106510000A8
:1006520031384632364B32302070726F746F202040
:010662000097
:1006630050696331384632364B323020657420434B
:0C0673004F473136204C4344200A0D0054
:020000040030CA
:0D00010002181EFF8980FF0FC007E00F40AE
:00000001FF
